:0200000480007A
:10000000971000009380000137513412130181676B
:100010009701000093810101678001001301000036
:1000200023A0000023A2200097100000938000FF6F
:100030001301F0FF9301F0FF37D2ED0F130292BAD4
:10004000970F0000938F8F0367800F00130100004C
:100050009301000013020000B741658793811132BC
:100060009702000093828203678002001301000060
:10007000930100001302000037E1BC9A130101EF65
:1000800097070000938787FD678007001301000032
:10009000930100001302000023A0000023A220000F
:1000A00023A4300023A6400097140000938484F515
:1000B00017150000130585F71301F0FF9301F0FFFA
:1000C0001302F0FF9302F0FF3753555513035355B6
:1000D00083AC040003AC4400970300009383430304
:1000E000E7800300B7212222938121221704000018
:1000F00013040404E70F0400B742444493824244CB
:10010000170F0000130FCF0467000F0037111111F4
:10011000130111116780000013010000930100001A
:100120001302000093020000130300003732333340
:100130001302323367800F001301000093010000A7
:10014000130200009302000013030000B3C39001E8
:1001500033C48F01232025002322350023244500AA
:100160002326550023286500232A7500232C8500AB
:1001700097140000938484E9171500001305C5EC5B
:100180001301F0FF9301F0FF1302F0FF9302F0FF61
:100190001303F0FF03AC040083AC44009707000096
:1001A0009387C70267800700B7717777938171776C
:1001B00067801F001301000093010000130200007C
:1001C0009302000013030000376166661301616645
:1001D000970F0000938F9FFDE78F0F00379288885D
:1001E000130282889700000093801002E7800000CD
:1001F00037B3AAAA1303A3AA170F0000130FCF0245
:1002000067000F00B7A299999382929967801000B6
:10021000130100009301000013020000930200008C
:1002200013030000B3C38F0133C4900123202500C2
:10023000232235002324450023265500232865006A
:10024000232A7500232C850097100000938080E1FD
:100250003712111113021211970100009381F1005E
:100260006780110013020000B7222222938222220B
:1002700097010000938111016780F1FF9302000054
:1002800037333333130333339701000093811181E4
:100290006780F17F13030000B743444493834344D2
:1002A0009711000093810181678001809303000012
:1002B00023A0400023A2500023A4600023A67000C6
:1002C00017150000130505D597150000938585DAED
:1002D000370610F01306C6F26306B5028326C50082
:1002E0002320D600832685002320D60083264500C0
:1002F0002320D600832605002320D6001305050100
:100300006FF09FFD370510F0130505F2232005005F
:0403100000000000E9
:10100000E4000080F8000080DC010080F001008036
:10101000FFFFFFFFFFFFFFFFFFFFFFFFFFFFFFFFE0
:10102000FFFFFFFFFFFFFFFFFFFFFFFFFFFFFFFFD0
:10103000FFFFFFFFFFFFFFFFFFFFFFFFFFFFFFFFC0
:10104000FFFFFFFFFFFFFFFFFFFFFFFFFFFFFFFFB0
:10105000FFFFFFFFFFFFFFFFFFFFFFFFFFFFFFFFA0
:10106000FFFFFFFFFFFFFFFFFFFFFFFFFFFFFFFF90
:040000058000000077
:00000001FF
